:060000000F308A00002809
:1010000003138316203099000D2803138312A101C6
:1010100083168B138B1B052812288312A101A114A0
:101020008316181518080439223898000F308A00E2
:1010300007178717D7308100831290309800C601B8
:10104000C501A001C0014014A42600261426A01C3E
:101050002F28A11C2F286E234B21201D7C28A01790
:101060008220A013201B3728A0187C282F283B267D
:101070006E236F210008B621AC00031938285730C1
:101080002C02031D4528D620382852302C02031D7F
:101090004B28A5203828840A0008031D7A283F30F1
:1010A0002C02031D55288D25382855302C02031D90
:1010B0006628A222201D3828A01962286C25042148
:1010C000142638283F2196232D25382844302C0219
:1010D000031D6C28CC21382851302C02031D7428A4
:1010E000A0187C281426382856302C02031D7A2894
:1010F00014263828AA243828A01C38285E260E304A
:101100008A00FC2E2013A3285030A0216130A0219A
:101110007330A021A0217730A0216F30A021723040
:10112000A0216430A0213E30A0216F212208F627A3
:101130000002031DA42800080319A328A219A4284B
:10114000A20A840A962820170800840A2030000288
:10115000031DBD28840AA011A721A800A019BD283D
:101160000008031DBD28A81FBA28A5012808A6004D
:10117000502408003124BF200800AA2408002808B1
:10118000CB202030A0213D30A0212030A0212708F5
:10119000CB2096230800B900F039B000300EE527C7
:1011A000A02139080F39E527A0210800840A203042
:1011B0000002031D0229840AA011A721A0190229F7
:1011C000A70020300002031D0229840A40300002DB
:1011D000031D0229840A20300002031D0229840A0B
:1011E000A721A800A81FF928A5012808A6005024B7
:1011F0000800A01902290008031D02291124312426
:10120000BF200800AA2408000F30A500C530A600A2
:101210003430A30058256F21A20A0008A400A2239D
:10122000000803190800A60A840AA20AA21A80016B
:101230000D296400201018192129981C232918123F
:1012400018161A0808008C1E080020141A08C3007B
:101250000A3C031920104308080081010B111921D1
:10126000201C332908000B1D2F29A1190800C50ACD
:101270000319C60AC61E0800A0187C280800A1157C
:101280002D2120183F292D2120183F292D212018FC
:101290003F29A11108002011A1150F30BE000F3009
:1012A000AB002030A021AB0B51293C30A0211030E5
:1012B000AB000830A021AB0B59290F30AB002D211A
:1012C00020186B29BE0B5F290F30BE002330A021F0
:1012D000AB0B5F296C292015A11196230800503013
:1012E0008400C601C5012D21201C7329083043024A
:1012F000031D892950300402031971298403083021
:10130000211CA0212030211CA0210830211CA0215B
:1013100071290D3043020319992943088000A01B4D
:101320002A30211CA0217F30040203199929840A44
:101330007129211C96238001A201503084000800ED
:1013400081010B1164000C1EA229990008000008FD
:10135000B6218C26A0190800B000B00E840A00083F
:10136000B6218C26B0043008840A0800C3007B3004
:1013700043020318C22961304302031CC2292030F2
:101380004302080043080800FB233F302302031DEB
:101390000800FF3024020800A0111426A01C080039
:1013A000A501A601B101C421031DDD29A60A031967
:1013B000A50A3D24A01DD229F8292508BA0026082F
:1013C000BB00B10A2608AF00A60A0319A50A2F0818
:1013D0002606F839031DF2293D24A019F729C42156
:1013E000031DE12930223D24A019F829D2293022F9
:1013F0000822A0113A30A0210030CB200030CB20B1
:101400000030CB200130CB20FF30CB2096230800CA
:10141000A8014230BF003A30A0211030B200B6001F
:101420000310B60CCB200310280D03183F143F08FF
:10143000B207CB200310280DB207CB200301CB202D
:1014400031242708B207CB200301CB20A80AB60B12
:10145000202AB209320ACB209623A81F0B2A0800A3
:101460003A08A5003B08A6003A30A0210310310D30
:10147000B200CB20260D250DB207CB200310260D80
:10148000B207CB200301CB20FB23A60A0319A50A30
:101490002408B207CB202308B207CB20B10B442A83
:1014A000B209320ACB20962308004530A0217230C1
:1014B000A0216130A0217330A0216930A0216E30BD
:1014C000A0216730A0219623A010A5010330A6001B
:1014D0003F30A300FF30A400A223A0190800A60AF1
:1014E000031D752AA50A2330A0213D24A01D6C2AC6
:1014F000A0110F30A500C530A6003430A300A40110
:10150000A223A0190800A60AE5302602031D802A9E
:101510000E30A500FC30A6003F30A300FF30A40031
:10152000A223A0190800A60A031D902A7F30A80054
:10153000FF30A7001124A0190800A80B9A2A112433
:1015400096230800A0112011B301B401B501413068
:10155000A0217230A0216530A0212030A021793057
:10156000A0216F30A0217530A0212030A021733040
:10157000A0217530A0217230A0216530A0213F301C
:10158000A0212030A0215B30A0217930A0212F3074
:10159000A0214E30A0215D30A0213E30A0216F213E
:1015A0000008B621593C031D0800840A0008031DE9
:1015B000080020155522A01908005230A0216530DE
:1015C000A0216130A0216430A0217930A021962390
:1015D000211621146F212110B30A0A303302031C93
:1015E000F92AB301B40A0A303402031CF92AB401FF
:1015F000B50A00083A3C031D512B840AA721A01903
:101600000800B100B2000310310CB100B800A721EE
:10161000A0190800A500B207A721A0190800A6007C
:10162000B2070310A50CA60CA721A0190800B7004B
:10163000B207B708031D4D2B0408C200B1080319F7
:101640002B2BA721A0190800B207A721A019080079
:10165000B207B1031E2BA721A0190800B207031D72
:10166000642B42088400B808031D392B2330A021C5
:10167000E92AA721A400A721A3003D24A0195024F2
:10168000A0190800A01EA223A01A6823A019080010
:10169000A60A0319A50AB803332B962337030319A7
:1016A000542BA015E6240800A721A0190800B207B2
:1016B000031D642B0026A0180800A0157723B30192
:1016C000B401B501B30A0800A0159623002508004F
:1016D0002408A7002608A800112408005030A021E3
:1016E0004930A0214330A0213E30A02108003030F5
:1016F000A021A021A0213230A0216830A0212030DB
:10170000A0212130A0213D30A0212030A021673030
:10171000A0216F30A0217430A0216F30A021203093
:10172000A0215830A021A021962308000A30A02132
:101730000D30A02108002030A0212D30A021203024
:10174000A02108002012640020302502031908009F
:101750002508C7002608C8002508031DB72B03303D
:1017600026020318B72B0E30A500FC30A60725086B
:1017700003178F000313260803178D000313230894
:1017800003178E000313240803178C0083168C178D
:101790000C1555308D00AA308D008C14FF3FFF3F93
:1017A000FF3FFF3FFF3FFF3FFF3FFF3FFF3FFF3F49
:1017B000FF3FFF3FFF3FFF3FFF3FFF3F00000000B5
:1017C0000C110C140000000083120E0803132302F6
:1017D000031DF02B03170C08031324020319F62B27
:1017E000201AF42B2016B72B8D24A0154708A5002E
:1017F0004808A60008006400250803178F0003139B
:10180000260803178D0083168C170C1400000000A7
:1018100083120E080313A30003170C080313A4007C
:1018200008000D12280803178D000313270803175B
:101830008C0083168C130C1555308D00AA308D004A
:101840008C148312031364000D1E232C03178316BC
:101850000C110C1483120C0803132702031D9B2484
:1018600008006400280803178D0083168C130C14DD
:1018700083120C080313A7000800A01208302502E9
:10188000031C08002508203C031908002508213CFA
:10189000031D4E2CA61B4E2CA0160800A0150800F8
:1018A0004D30A0216530A0216D30A0216F30A021E6
:1018B0007230A0217930A0212030A0217030A021E9
:1018C0007230A0216F30A0217430A0216530A0219A
:1018D0006330A0217430A0216930A0216F30A02195
:1018E0006E30A0211325212508002030A021703062
:1018F000A0217230A0216F30A0216730A02172306A
:10190000A0216130A0216D30A021A0216930A0214B
:101910006E30A0216730A02108004630A0214C3055
:10192000A0214130A0215330A0214830A0217524AE
:101930001325212508004530A021A0215030A021E9
:101940005230A0214F30A0214D30A0217524962384
:10195000A0150800D5246330A0216F30A0216D3080
:10196000A021A0216130A0216E30A0216430A021EF
:10197000962308004E30A0216F30A0216E30A021A8
:101980002D30A0214830A0214530A0215830A02181
:101990002030A0216330A0216830A0216130A02137
:1019A0007230A0211325962308004930A0216E3003
:1019B000A0217630A0216130A0216C30A0216930B7
:1019C000A0216430A0212030A0210800D52472304D
:1019D000A0216530A0216330A0216F30A02172309A
:1019E000A0216430A0212030A0217430A0217930C2
:1019F000A0217030A0216530A02113259623080076
:101A00004330A0216830A0216530A0216330A0219F
:101A10006B30A0217330A0217530A0216D30A02142
:101A20001325962308002030A0216530A0217230B4
:101A3000A021A0216F30A0217230A0212030A02150
:101A400008004030A0212030A0212508CB20260806
:101A5000CB206830A021962308004C30A0216930AB
:101A6000A0216E30A0216530A0212030A0216E3051
:101A7000A0217530A0216D30A0216230A0216530F9
:101A8000A0217230A0212030A021A0123508031916
:101A90004C2DA016E527A0213408A01A512D0319BA
:101AA000532DE527A0213308E527A0219623080020
:101AB0004530A0216E30A0217430A0216530A021D6
:101AC0007230A0212030A0216130A0212030A0213F
:101AD000CB253E30A02108005530A0217030A02138
:101AE0006C30A0216F30A0216130A0216430A02192
:101AF0002030A0217330A0217530A0216330A021B7
:101B0000A0216530A0217330A0216630A02175305E
:101B1000A0216C30A02196230800C001C014A42687
:101B2000752696235530A0219B235530A021703077
:101B3000A0216C30A0216F30A0216130A021643041
:101B4000A02175267430A0216F30A021E0254430FB
:101B5000A0219B234430A0216F30A0217730A02109
:101B60006E30A0216C30A0216F30A0216130A02107
:101B70006430A02175266630A0217230A0216F301C
:101B8000A0216D30A021E025C0014015A4267526B6
:101B9000CB25962308007230A0216530A021763035
:101BA000A0212030A0217330A0217430A0217230F8
:101BB000A0216930A0216E30A0216730A02108004B
:101BC0002030A0217030A0217230A0216F30A021E0
:101BD0006730A0217230A0216130A0216D30A0219A
:101BE0002030A0216D30A0216530A0216D30A021D2
:101BF0006F30A0217230A0217930A02196230800F7
:101C0000A0100E30A500FC30A600FB2323083839B5
:101C1000283A0319122EFE30A600FB232308383978
:101C2000283A0319A0140800A01C212EC527FF394B
:101C30000319332EC0014016A426C001C015A426E6
:101C4000392E4E30A0216F30A02175266C30A02196
:101C50006F30A0216130A0216430A0216530A02127
:101C60006430A021392E4E30A0216F30A02175267E
:101C7000CB259623080052263F30A0212030A021FA
:101C80006630A0216F30A0217230A0212030A02129
:101C90006830A0216530A0216C30A0217030A021D7
:101CA000962308005030A0217230A0216530A02179
:101CB0007330A021A0212030A02108004A30A021AB
:101CC0007530A0216D30A0217030A0216930A02195
:101CD0006E30A0216730A0212030A0217430A021D7
:101CE0006F30A0217526962308002030A021753082
:101CF000A0217330A0216530A0217230A0212030B6
:101D0000A0216330A0216F30A0216430A021653074
:101D1000A0212030A0210800AF003030AF02031C0A
:101D2000A12E0A302F02031C9F2E1130AF02031C7C
:101D3000A12E06302F020318A12E0A30AF072F085C
:101D40000800A015BA240034AF012F0840188C27D2
:101D5000C0185F2740190027C019C427401A4D2713
:0C1D6000FF3903190800A021AF0AA52ECE
:101E00008207573420342D342034573472346934E7
:101E100074346534203474346F342034453445349C
:101E2000503452344F344D342C342034223457340F
:101E30002034443444342034403420344134413458
:101E400022340A340D34523420342D3420345234A8
:101E50006534613464342034663472346F346D34E4
:101E6000203445344534503452344F344D342C34BE
:101E700020342234523420344134413422340A3460
:101E80000D34563420342D342034443469347334C2
:101E900070346C34613479340034820743347534DF
:101EA0007234723465346E347434203469346D3471
:101EB00061346734653420343D3420340034820783
:101EC0003F3420342D342034443469347334703436
:101ED0006C34613479342034743468346934733444
:101EE00020346C346934733474340A340D3451340E
:101EF00020342D3420345134753469347434203412
:101F000061346E34643420346A3475346D34703422
:101F1000203474346F34003482071B345B34323421
:101F20004A3434344B3420345034493443344C3400
:101F30004F344134443445345234203476343134CF
:101F40002E34333431340A340D34A93452342E341F
:101F50004634613472346D34653472342F34523403
:101F60002E345034653472346434723469346134DC
:101F70007534203431343934393439340A340D3439
:021F800000342B
:081F880082070034003400342C
:101F900000340034003400340034003400340034A1
:101FA0000034003400340034003400340034003491
:101FB0000034003400340034003400340034003481
:101FC00000340034003400340034820730343134BB
:101FD00032343334343435343634373438343934B5
:101FE000413442344334443445344634820748341F
:101FF00065346C346C346F343134323433340034FF
:02400E00323F3F
:00000001FF
